:100000006F00E06C00000000F2010000F60100004B
:1000100000000000000000000000000000000000E0
:1000200000000000000000000000000000000000D0
:100030009C060000000000009E060000000000007A
:10004000A0060000A2060000A4060000A60600000C
:10005000A8060000AA060000AC060000AE060000DC
:10006000B0060000B2060000B4060000B6060000AC
:10007000B8060000BA060000BC060000BE0600007C
:10008000C0060000C2060000C40600006E040000A6
:10009000C8060000CA060000CC06000000000000F0
:1000A000511126C022C206C4828282441244A24058
:1000B000310182802A86014593F6150091C232955E
:1000C00085810606F5F9828000000000634E050276
:1000D00063C305042E86AA857D5515C285466378BF
:1000E000B6006356C00006068606E36CB6FE014500
:1000F00063E4C500918D558D85820582F5FA828075
:100100008682C93F2E8582823305A04063D70500D1
:10011000B305B040C1B7B305B0408682653F330533
:10012000A0408282868263C70500634905005D376F
:100130002E858282B305B040E35B05FE3305A04007
:10014000513F3305B040828200003D432A876373EC
:10015000C3029377F700BDEFADE5937606FF3D8AC6
:10016000BA960CC34CC30CC74CC74107E36BD7FE10
:1001700011E28280B306C3408A0697020000969679
:100180006780A6002307B700A306B7002306B700C1
:10019000A305B7002305B700A304B7002304B700E5
:1001A000A303B7002303B700A302B7002302B700DD
:1001B000A301B7002301B700A300B7002300B700D5
:1001C000828093F5F50F93968500D58D9396050162
:1001D000D58D61B793962700970200009696868288
:1001E000E78086FA9680C1171D8F3E96E374C3F8A8
:1001F000A5B77300203001A0EFF29FEA11118545E9
:10020000116502C002C202C402C602C802CA02CC00
:10021000EF00F00E930700027C80371501408D47F8
:100220003EC28A85E147130505403EC4EF00006ADF
:10023000896737440140938707583EC66C00B7076B
:100240000800130504803ECA02C8231C0100EF0009
:100250003015854513050480EF0050217101B1B5BB
:10026000EFF21FE43715000031111305C53EEF1002
:10027000C00E0564130504808545EF005008214732
:10028000B7E700E023A2E7101304F49522C49967AE
:10029000373401409387871A2C00130504C03EC6EB
:1002A000EF00D00705468545130504C0EF00F00BAD
:1002B000930730127C8089475C810A8585473EC25E
:1002C000EF00806E835704C093E717002310F4C03B
:1002D0005101E1BBEFF2DFDC2111614681450A8566
:1002E000AD35854513050020EF0070013165EF0045
:1002F000007637240140B7070E003EC68A85854741
:1003000013050440230AF10002C002C202C402C85D
:1003100089219D4605469D4513050440C129B70521
:10032000000213050440492B8545130504408D291F
:1003300013050440B529930404402685BD2975FDA5
:100340001305044037240140AD29130404402285DD
:10035000B52975FD610191BBEFF29FD4511185451F
:10036000414502C002C202C4EF0060799307100742
:1003700009447C808A85C147371501403EC422C2AA
:10038000B123854513050002EF006077B7140140E3
:10039000214778808A856147138504403AC422C288
:1003A0003523C1478A85138504407C8022C202C45C
:1003B000312B3101DDB9EFF2BFCE37250140854544
:1003C0001305054037240140312193040440894539
:1003D0002685F1296DDD13050440F121F9B1EFF215
:1003E0003FCC371701405C47371500001305453BEC
:1003F00093E717005CC77D57A388E180EF00D073B7
:100400006DB1EFF2FFC9371701405C4737150000A7
:100410001305453AF99B5CC7A3880180EF00D071B2
:1004200069B1EFF2FFC70945AD2B1924EF00900623
:10043000716513050520EF00D00CB707002083A5D8
:1004400007013715000013050540EF00F06E6D330E
:1004500021374935313513054006EF00F006553791
:10046000F327003093E787087390073001A0371512
:10047000000051111305053C22C426C2EF00F06DA7
:10048000373501408545130505C0CD2D8547631CD3
:10049000F50613054006EF00300383C701810D47C1
:1004A00093840181850793F7F70F6389E7069CA082
:1004B0003716014054469C203704002093F6F60876
:1004C00013974700558F3EC058C6F53582478C209C
:1004D000130484038607A2978AA393971500A29713
:1004E0009223371500001305453DEF00F06403C764
:1004F00011819C20860715E73E941A2093077039D6
:1005000063F3E700E93D373501408545130505C034
:10051000512522449244310173002030238004008D
:1005200041BFA2979A239307C035E3EEE7FCD13D84
:10053000D9BFB71702409843B706FFFC6111136794
:10054000170098C3D8432166758FD8C39843B70660
:10055000F7FEFD16758F98C39843B706FCFFFD168E
:10056000758F98C3D843C176FD16758FD8C33707EA
:100570009F0098C702C002C2984FB7060140136798
:10058000170098CFD842518FD8C29843C16637061A
:100590000200558F98C3B716024009679C42F18F3D
:1005A0003EC2824785073EC0924781E78247E39774
:1005B000E7FEB71702409C431397E700635807060E
:1005C00085473EC2124785476310F706B7270240AA
:1005D0009843C176FD16719B98C398431367170023
:1005E00098C3B7170240D843D8C3D843758FD8C330
:1005F000D843C166558FD8C39843B7060001558FBD
:1006000098C3984393166700E3DD06FED843B716F8
:100610000240719BD8C3D84313672700D8C3214732
:10062000DC42B18BE39EE7FE2101828002C259BF0A
:10063000EFF21FA7371702405C43370400209146B2
:10064000B18B130404016385D700A1466380D704EE
:10065000B7376E01938707601CC0B7160240DC42B3
:100660000840918313F7F700B7070020938707002E
:10067000BA978C23DC4293F5F50F93F707083357AD
:10068000B50099E3813C2A8718C005B45C43B7776D
:10069000DC02938707C0C9B701A001A001A001A097
:1006A00001A001A001A001A001A001A001A001A042
:1006B00001A001A001A001A001A001A001A001A032
:1006C00001A001A001A001A001A001A001A097012B
:1006D00000209381A116138181FC171500001305DA
:1006E000E5D3970500209385E591170600201306B2
:1006F000E69463FAC5008322050023A05500110586
:100700009105E3EAC5FE170500201305259393859F
:10071000C1816377B500232005001105E36DB5FEA7
:1007200093020008739002308D42739042809702CA
:1007300000009382228D93E2320073905230EFF0EA
:100740005FDF97020000938202CE73901234730031
:1007500020305C413707F1FF1307F7EF7D8FDC4155
:100760009441A207D58FD98F5CC11C4537F7F1FFA3
:100770001307D77FD4457D8F9C49D58F9445860636
:10078000D58FD98F1CC55C55370710FF7D177D8F1E
:10079000DC29FD1793F7F70FD207D98F5CD582803C
:1007A0001C4589C593E717001CC58280F99BEDBFE6
:1007B0001C4593E787001CC5828008450D8105898B
:1007C00082801C4593E747001CC58280084509814B
:1007D000058982801C4591C537075000D98F1CC5FB
:1007E00082803707B0FF7D17F98FD5BFA54763F823
:1007F000B704138765FF931717008322C500BA97C4
:100800001D433313F3001343F3FF33735300B397C4
:10081000F600B3E767005CC5994763E3C7047D163C
:10082000931726003E965859FD47B397C70093C7C4
:10083000F7FFF98FB395C500DD8D4CD98280939772
:10084000150003230501AE971D473317F700134723
:10085000F7FF33776700B397F6005D8F18C96DBF58
:10086000B14763E2C7026516931726003E961859F2
:10087000FD47B397C70093C7F7FFF98FB395C5003E
:10088000DD8D0CD982804D161317260054553A96EB
:10089000FD47B397C70093C7F7FFF58FB395C50022
:1008A000DD8D4CD5828068454205418182800841BA
:1008B0006D8D3335A00082805C41370700FA7D17CB
:1008C000F98F5CC15C41DD8D4CC182809C4561111A
:1008D00022C226C013F7070113F3F70001C7D8415E
:1008E0003363E30092211377F60F29C783230500B2
:1008F000014713048002930480048546B395E60003
:10090000B376B6006392D50293122700BD46B39624
:10091000560093C6F6FFB3F37600B3125300B3E369
:100920007200639787064CC90507A146E317D7FCF9
:10093000232075001307F00F6378C7048323450055
:10094000A14613048002930480040547B312D70024
:10095000337756006394E202139726000117BD45D2
:10096000B395E50093C5F5FFB3F375003317E300C6
:10097000B363770063928702232A550085064147B7
:10098000E395E6FC23227500124482442101828013
:10099000E39C97F80CC949BFE39297FE23285500C2
:1009A000F1BF23AAA18082809387418194431821BB
:1009B00081E63C21920721A894430546639FC60225
:1009C0003C21103192076314D60093E707F8B7E68D
:1009D00000E093F7F70FBA962380F64085469357C9
:1009E00057003397E6005441A5C2938707048A074E
:1009F000B7E600E0B69798C382808C43894663913E
:100A0000D50214313C216365D6008A06B6975DB7DE
:100A10009386E6038A06B69793F7F70F920775B7A2
:100A200090438D46631CD60014313C216364D6008C
:100A30008606E9BF9386C6078606F1BF94439147B1
:100A4000E39EF6F81C31BDB7938707064DB7B7167E
:100A50000240DC4241771307F77FF98F5D8DC8C2F2
:100A60008280EFF2EFE3371702405C4391462A841D
:100A7000B18B6385D700A146638DD706B7376E016A
:100A8000938707601CC0B7160240DC42918313F7BE
:100A9000F700B707002093878702BA978C23DC42C0
:100AA000184093F5F50F93F707083355B70081E722
:100AB0003A85EFF02FE248C008C448C4B717024097
:100AC000DC43AD83FD8B13D737008A07F18BD98FB9
:100AD00093F637010D476373D700D117370700200E
:100AE00013074701BA978C23EFF0CFDE08C86FF0E9
:100AF000CFDB5C43B777DC02938707C061B799C54A
:100B0000371702401C4F5D8D08CF8280B717024017
:100B1000984F1345F5FF798D88CF82801E21373796
:100B20000140130707C0C207C1836306E50037070A
:100B300000406316E500BA2193F7F7F8D98FFA2140
:100B400093F7F7CFC207C183D98F1EA1DE215EB50F
:100B50009E211EB5B7370140938707C06314F50087
:100B60009C251EB985475EA982805E2501C6DD8D64
:100B70004EA5828093C5F5FFFD8DDDBF1E294A2558
:100B8000ED8F4205418189C76D8D3335A00082808C
:100B90000145828093C5F5FFC205C1810EA98280FF
:100BA000EFF20FD01629F577FD17F58FF621DA252C
:100BB0002111D58F1EA95625FD779387379FF58F75
:100BC000D6212A842EC0D58F9625D58FB625D58FD0
:100BD0005EA55E29C207C18393F7F7CF5D8F5AA93F
:100BE00048004135B747014093870780824563122B
:100BF000F406C2475A24139517003E9542070E0586
:100C000041873E958C41635807048605EFF08FCCF1
:100C1000930540062AC0EFF0EFCB824793144500BE
:100C2000930540063E85EFF0AFCD5E24C207C18735
:100C300063D507020E059305400613052503EFF063
:100C40006FC91D89C98CC204C18006A461016FF0FF
:100C5000CFC5B24745B78A0555BF12059305400673
:100C600013052503EFF00FC73D89E9BF91C55E2548
:100C70000967D98F5EA582805A25F977FD17F98F0C
:100C8000D5BF93F5F51F4EA182800A216D8D3335B6
:100C9000A0008280EFF2CFC0B707002003A50701B4
:100CA000B7157A0093850520EFF0CFC21375F50FC5
:100CB000238DA18093175500898F8A073E950E05D5
:100CC000239CA1806FF06FBEEFF28FBD37F400E080
:100CD0005C40AA85F99B5CC003D58181EFF08FBD94
:100CE00008C8232404001C4093E717001CC0B7F772
:100CF00000E0D843058B75DF9843799B98C36FF06C
:100D0000CFBAEFF2EFB92A841165111185451305A9
:100D10000502F533930700027C80371501408D47AB
:100D20003EC28A85E147130505403EC4453622C6CA
:100D300037440140B70708006C00130504803ECA21
:100D400002C8231C0100A93D854513050480393FD5
:100D500071016FF08FB5EFF2AFB47111AE84014441
:100D6000635DC402B7470140138707803A85930546
:100D7000000432C0193FB74701401387078002467D
:100D800075D5338784008305070013850780050424
:100D9000C205C181FD350246E1B7328511016FF010
:100DA000CFB0411106C62EC00DCD1841AA8705C38C
:100DB00058417D5511CB8546631BD70098472300CA
:100DC000070023A207000545B240410182809847F1
:100DD000824614A39847050798C7D8437D17D8C300
:100DE000DDB705468A85853FF9BF011122CC2EC2A9
:100DF00006CE26CA2A84814793050002634506026F
:100E00009245BE95838505008DE563D8C70263D4FE
:100E1000E702198E1305000293F526002AC089C542
:100E200001E7930500032EC0858A814495EAB284C8
:100E30000DA08507F1B71D8EF1BF0146E1BF8245C8
:100E400022853AC832C63EC4A93FA247324642472D
:100E5000FD14E34690FEB284635306008144058E80
:100E600063C7E702A6879246338797403697830584
:100E7000070095EDB2846344900463530600014675
:100E8000F2406244D2443305F600056182801D8F32
:100E9000BA8793050003228532C83EC63AC411378B
:100EA000B24722474246FD17EDF7BA9465BF228547
:100EB00032C63EC4FD35A247324685076DB782452E
:100EC000228532C43EC2F13DFD142246924765B7E9
:100ED000397106DE22DC26DA3EC232833A8689ED9B
:100EE00092469307000301476C08FC86FD3DF250D3
:100EF0006254D25421618280AA843684AE8791CA1A
:100F0000294701446317E30063D50500B307B040E8
:100F100005448646A309010213073103938666FC44
:100F200036C49A853E8532CA3AC81AC63EC0EFF02A
:100F30002F9DA546824732434247524663D4A600BE
:100F4000A2463695130505039306F7FFA30FA7FEE8
:100F50009A853E8532CC3ACA1AC83EC636C0EFF0F2
:100F60006F97B24742435247624663F9670401CC28
:100F700029CA9247898BB1C79305D002268532C40E
:100F80000D3522467D169247918B95C306479307F0
:100F9000100632C4930500032685631EF70211353F
:100FA000930580072685F53B2246090479161647E6
:100FB000924682452685153D229515BFAA87024790
:100FC0008DB782469307D0020144A38FF6FE9307A4
:100FD000E7FF3EC04DBFF13393058005E1B7014502
:100FE000828001458280130181FD22D026CE06D267
:100FF0002AC4AE82328402C681448385020089ED10
:10100000A24781C781453E85693B9250025426859F
:10101000F244130181028280930750026388F50035
:10102000224516C88504B53BC24239A88387120001
:1010300013871200639CB7002245930550023AC8FB
:101040008D3342478504BA82850245BFD5DB9306BE
:10105000B0026389D70463C8F60093063002638642
:10106000D704814705A09306D002638AD700930670
:101070000003E398D7FE13872200894721A0138736
:1010800022008547830607001306B0026383C60467
:101090006341D60213063002638BC602BA82014551
:1010A000A54681A0138722006DBF138722009147B8
:1010B000D1BF1306D0026389C60013060003E39F65
:1010C000C6FC93E7270031A005078547C1BF93E71A
:1010D00047000507E1B713162500329506053A9536
:1010E000850203860200130706FD9375F70FE3F4EC
:1010F000B6FE1307E0029946631EE60085028146AC
:10110000A54503860200130606FD1377F60F63F567
:10111000E50236C6038702001306A006630DC70A60
:101120006343E6021306C0046307C70A130680067A
:10113000630CC70881452DA813972600BA9686062A
:10114000B29685027DBF130640076306C7081306E3
:10115000A0076302C7081306C0068145631AC700CB
:10116000038612008D456314E600850291458502D1
:1011700003860200930300061307100663C4C3002E
:10118000130710049303700663C4C3069303500649
:10119000635376189303700463C1C304930550042A
:1011A000635BB61613073004E310E6EA18409303B6
:1011B000440016CA230CE1001EC8A30C010001471D
:1011C000BE862A862C0849A8038612008145E311B1
:1011D000E6FA890271BF8502B1BF93063006E307C4
:1011E000D6FC63CEC606930680056303D602A9BD6E
:1011F000930630076304D60463CBC6029306F00659
:101200006302D60E9306000793E74700E31ED6E27B
:101210009146639FD50A930384000C40504016CA40
:101220003AC23EC01EC8AA870147C146B9A093066C
:1012300050076308D6069306800745BF1840B716C7
:101240000000930344009385064111C3BA853247D9
:1012500016CA1EC8BE862A862245413E0DA091466A
:101260006394D502930384000C40504016CA3AC2DE
:101270003EC01EC8AA870547A94622458D33C243F2
:10128000AA941E84D242C9B3B2460C4016C836C2D4
:101290003AC011042A878546294622451539AA9461
:1012A00061B39146639DD500930384000C40504088
:1012B00016CA3AC23EC01EC8AA87014775BFB246C9
:1012C0000C4016C836C23AC011042A878146E9B7D5
:1012D000B24616C80C40414636C23AC011042A87AD
:1012E000814665BF9146639ED500930384000C4000
:1012F000504016CA3AC23EC01EC8AA870147A1463E
:10130000ADBFB2460C4016C836C23AC011042A8797
:101310008146214659B70C401306840040403AC22A
:101320002A87224532C83EC02286B687A94616CAF9
:101330004D39AA944244B9B71301C1FD2EC832CA2F
:10134000AA851008014506C636CC3ACE3ED032C03A
:101350005939B240130141028280411122C426C290
:1013600006C61C21AA840144DC81830731000504E0
:1013700099EFA9479305310005460145DC81EFF05F
:101380009F9D2285B24022449244410182800546BD
:10139000930531000145EFF01F9CB38784009C2327
:1013A000DC81E1B7486561746572204F66660A0D9D
:1013B00000000000486561746572204F6E0A0D00E0
:1013C00054696D657220696E746572727570740D02
:1013D00000000000414443206368616E6E656C202C
:1013E0002564203D2025640D0A00000054696D65C8
:1013F00072204346472073746172740D0000000030
:1014000053797374656D436C6B3A25640D0A000063
:08141000286E756C6C290000C8
:10141800010203040506070801020304050607087C
:10142800006CDC020204060804080C1008101820DE
:1014380010203040204060800102030405060708A0
:08144800010203040506070878
:00000001FF
